:1000000012C084C0189518951895189518951895CC
:100010001895189518951895189518951895189578
:100020001895189518958FED8DBFC8EBE0EA4E2E08
:10003000DD275D2EA89584B7082E877F84BF88E1D1
:10004000992781BD91BDEEE7F0E0A0E6B0E08827FA
:100050008D933197E9F766248FEF87BB8FEF81BBD4
:10006000829A83E08093690084E080936A0085E04F
:1000700080936B0086E080936C00E0E0F0E0A1E606
:1000800045D1E1E0F0E0A2E641D1E2E0F0E0A3E614
:100090003DD1E3E0F0E0A4E639D178947BB7706419
:1000A0007BBF7FEF72BB70E078BB81E08093600024
:1000B00000916000043010F009F025C0A0E6AD907A
:1000C000A4E6AA0D8C9188BBA0E6AD90A8E6AA0D87
:1000D0008C91A2E3FFD0F4D08C9189238C9381E0A2
:1000E00090E0CCD0A0E6AD90A8E6AA0D8C91A2E35A
:1000F000F1D0E6D09C91982B9C93A0E68C918F5FD9
:100100008C9308F4D5CFD1CFF894FFCF0F921F92E4
:100110002F923F924F925F927F92AF92BF920F9336
:100120001F932F933F934F935F936F937F938F937F
:100130009F93AF93BF93CF93DF93EF93FF938FB7CB
:100140008F937FEF72BB829901C0FDCFA2E68C91A5
:100150008F5F8C9300916100093010F009F001C0AD
:1001600007C0A2E68C918F5F8C9380E08093610042
:1001700000916200093010F009F001C007C0A3E649
:100180008C918F5F8C9380E080936200009163007C
:10019000093010F009F001C007C0A4E68C918F5F10
:1001A0008C9380E08093630000916400093010F02C
:1001B00009F001C003C080E080936400E0E0F0E05B
:1001C000A1E67BE792D0E1E0F0E0A2E67BE78DD00C
:1001D000E2E0F0E0A3E67BE788D0E3E0F0E0A4E62D
:1001E0007BE783D0E0E6F2E0A1E68C919927A5E6D3
:1001F00064D0E0E6F2E0A2E68C919927A6E65DD015
:10020000E0E6F2E0A3E68C919927A7E656D0E0E677
:10021000F2E0A4E68C919927A8E64FD08AEF90E00F
:100220002DD0829901C0FDCF8F918FBFFF91EF91AB
:10023000DF91CF91BF91AF919F918F917F916F91FE
:100240005F914F913F912F911F910F91BF90AF9070
:100250007F905F904F903F902F901F900F90189538
:100260007B09E3CB99DAFA0BFBDB3197F1F70895C1
:10027000689462F80895E89462F80895EF93FF9304
:10028000EE27E82BE92B31F0E0EDF7E03197F1F7BD
:100290000197D1F7FF91EF910895C895319600200D
:1002A000089591E005C092E003C094E001C098E099
:1002B000F4DF0D929A95E1F70895E80FF91FF1CF59
:1002C00091E0882321F08894991F8A95E9F7892F76
:1002D00090950895883018F011968850FBCF0895B6
:1002E000E199FECFEEBB3196089591E001C092E016
:1002F0007B3751F47FB7F894F3DF8D918DBBE29A91
:10030000E19A9A95C9F77FBF7727089591E001C0D8
:1003100092E0E6DFE09A8DB38D939A95D1F7089538
:00000001FF
